:020000040000FA
:1000000039EF00F0FFFFFFFF4582E1CF15F0E2CFAF
:1000100016F0D9CF17F0DACF18F0F3CF19F0F4CFEC
:100020001AF0F2AC18D00E01C0B1C8A103D03CEC5C
:100030000BF011D0C0B9C8A903D0B2EC15F00BD0A9
:10004000C0BBC8AB03D098EC12F005D0C1B7C9A7AC
:1000500002D0AEEC16F01AC0F4FF19C0F3FF18C0BE
:10006000DAFF17C0D9FF16C0E2FF15C0E1FF4592C5
:100070001100ECEF11F051EC16F0F28EF28C829040
:10008000AFEC11F0C2EC10F0B9EC0EF07A0E0101F9
:10009000F06FC10EEF6F810EE82EFED7EF2FFCD769
:1000A000F02FFAD700D0A8EC16F0290E0101F06F5E
:1000B000960EEF6F7F0EE82EFED7EF2FFCD7F02FB6
:1000C000FAD78280C8EC16F0C6EC16F0010E1F6E4F
:1000D000010E206E460E61EC14F0010E1B6E750EC3
:1000E000EBEC13F0010E1B6E6E0EEBEC13F0010E39
:1000F0001B6E6B0EEBEC13F0010E1B6E2D0EEBEC7A
:1001000013F0010E1B6E530EEBEC13F0010E1B6E81
:10011000630EEBEC13F0010E1B6E610EEBEC13F0B3
:10012000010E1B6E6E0EEBEC13F0410E0101F06F31
:10013000F00EEF6F330EE82EFED7EF2FFCD7F02F27
:10014000FAD7010E0201836F930E8325D96EDA6A06
:10015000000EDA22DF50D8B4A2D0930E8325D96ED8
:10016000DA6A000EDA22DF500001F56F210EF66F19
:10017000000EF76F9F0E02018325D96EDA6A000E1A
:10018000DA22DF5083EC0CF00A0E0001A86F78D061
:10019000F3EC14F00001CB05D8A472D0400E611925
:1001A000D8A404D00A0EA86F000ECB6F810E61197F
:1001B000D8A466D0000E02017A6F27EC12F0000E70
:1001C0000001A86F000ECB6F9F0E02018325D96E30
:1001D000DA6A000EDA22B10E0001AE25E16EE26AA3
:1001E000010EE222DFCFE7FFAE51D8A431D0010EDD
:1001F0001F6E010E206E480E61EC14F0010E1B6E96
:10020000520EEBEC13F0010E1B6E580EEBEC13F0DC
:10021000010E1B6E200EEBEC13F0010E1F6E070E8D
:10022000206E200E61EC14F0010E1B6E200EEBEC24
:1002300013F0010E1B6E200EEBEC13F0010E1B6E83
:10024000200EEBEC13F0010E1B6E200EEBEC13F006
:100250000001AE51030DF350050F02017A6F010E3C
:100260000001FB6F7AC2FCF09F0E02018325D96E5C
:10027000DA6A000EDA22DF503AEC14F00001AE2BFD
:10028000A851D8A485D7290E0101F06F960EEF6F03
:100290007F0EE82EFED7EF2FFCD7F02FFAD7020102
:1002A000832B040E836550D7010E0001B46F000E3E
:1002B000386E000E346E41EC16F0190E0101F06F2D
:1002C0005A0EEF6FB10EE82EFED7EF2FFCD7F02FAE
:1002D000FAD700D0A8EC16F0290E0101F06F960EA7
:1002E000EF6F7F0EE82EFED7EF2FFCD7F02FFAD757
:1002F000010E1F6E010E206E430E61EC14F0010E14
:100300001B6E440EEBEC13F0010E1B6E5A0EEBEC61
:1003100013F0010E1B6E200EEBEC13F0010E1B6EA2
:10032000480EEBEC13F0010E1B6E520EEBEC13F0CB
:10033000010E1B6E200EEBEC13F0010E1B6E200E57
:10034000EBEC13F0010E1B6E3A0EEBEC13F0020E09
:100350001F6E050E206E480E61EC14F0010E1B6E30
:10036000520EEBEC13F0010E1B6E200EEBEC13F0B3
:10037000010E1B6E200EEBEC13F0010E1B6E3A0EFD
:10038000EBEC13F0F3EC14F00001A751D8A42BD040
:10039000990EA76F000E396E3850D8B418D0220EBF
:1003A0003824D96EDA6A000EDA22DFB010D0220EBD
:1003B0003824D96EDA6A000EDA22000EDF6E870E5C
:1003C0003824D96EDA6A000EDA22000EDF6E7CEC79
:1003D00016F0386E0F0E3818D8B403D0040E396EEC
:1003E00002D0000E386E0001CB05D8A40DD027EC4A
:1003F00012F00201796F000E0001CB6F220E1B6E0E
:100400000201795119EC0EF00001C351D8A415D0A6
:10041000990EC36F000E346E010E02017E6F040E42
:100420007E6501D00AD0E10E7E25D96EDA6A010E12
:10043000DA22000EDF6E7E2BF2D73450D8A44FD0D4
:100440000001AB51D8A44BD0030EAB6F040E356442
:1004500003D0010E356E01D0352A3950D8B426D0DC
:1004600039A616D0930E3824D96EDA6A000EDA2235
:10047000DF50F56F2F0EF66F000EF76F9F0E3824CA
:10048000D96EDA6A000EDA22DF5083EC0CF00BD062
:1004900039A409D0000EF56F2E0EF66F000EF76F1F
:1004A000000E83EC0CF0000E396E19D03550D8B424
:1004B00016D0930E3524D96EDA6A000EDA22DF5098
:1004C000D8B40DD035500C0D000EF324D96E020EA9
:1004D000F420DA6E000EDF6E35504AEC0FF0010E9C
:1004E0000201846F040E846501D03DD0220E842564
:1004F000D96EDA6A000EDA22DFA033D07B0E8425B3
:10050000D96EDA6A000EDA22040EDF642AD0000EF9
:10051000786F7B0E8425D96EDA6A000EDA22000E1F
:10052000DF6E3B0E8425D96EDA6A020EDA22000EE7
:10053000DF6E220E8425D96EDA6A000EDA22000EF2
:10054000DF6E8D0E8425D96EDA6A000EDA22000E77
:10055000DF6E870E8425D96EDA6A000EDA22000E6D
:10056000DF6E842BBFD70001AA51D8A404D01E0E81
:10057000AA6F16EC15F00001A951D8A403D7000EFC
:1005800002017F6F140E0001A96F87EC14F00201C5
:100590007B6F0001BB05D8A4C3D0000EAC6FA605CD
:1005A000D8A405D0050E02017C6F010E7D6F020EEE
:1005B0000001A619D8A405D00D0E02017C6F010E12
:1005C0007D6F030E0001A619D8A405D0050E020107
:1005D0007C6F020E7D6F040E0001A619D8A405D011
:1005E0000D0E02017C6F020E7D6F220E0001A6250A
:1005F000D96EDA6A000EDA22DF50D8A428D0CF0EE6
:10060000A625D96EDA6A010EDA22DF50D8A4DDD130
:10061000CF0EA625D96EDA6A010EDA22010EDF6E40
:100620007DC21FF07CC220F0200E61EC14F0010EA0
:100630001B6E200EEBEC13F0010E1B6E200EEBEC8C
:1006400013F0010E1B6E200EEBEC13F0BED1CF0E9B
:10065000A625D96EDA6A010EDA22000EDF6EA651E7
:100660000E0D550EF324D96E010EF420DA6EDF5014
:100670000201826F0001A6510E0D560EF324D96EB1
:10068000010EF420DA6EDF5002017F6F0001A651E7
:100690000E0D570EF324D96E010EF420DA6E01010F
:1006A000DFAC02D0010E01D0000E0201806F00010C
:1006B000A6510E0D570EF324D96E010EF420DA6EFA
:1006C0000101DFAA02D0010E01D0000E0201816FEC
:1006D0000001A6510E0D570EF324D96E010EF42021
:1006E000DA6E0101DFA404D0020182513D0F826F56
:1006F00082C2E6F17FC2E7F1000E0101E86F000E51
:10070000E96F80C2EAF181C2EBF17DC2ECF17CC2FB
:10071000EDF1000EEE6F0001A65156EC10F055D130
:10072000AC51D8A442D0010EAC6F010E1F6E050E65
:10073000206E480E61EC14F0010E1B6E520EEBECB5
:1007400013F0010E1B6E200EEBEC13F0010E1B6E6E
:100750002D0EEBEC13F0010E1B6E200EEBEC13F0E4
:10076000010E1B6E200EEBEC13F0020E1F6E050E39
:10077000206E480E61EC14F0010E1B6E520EEBEC75
:1007800013F0010E1B6E200EEBEC13F0010E1B6E2E
:10079000200EEBEC13F0010E1B6E200EEBEC13F0B1
:1007A000010E1B6E200EEBEC13F0220E0001A625AD
:1007B000D96EDA6A000EDA22DF50D8A480D0CF0ECC
:1007C000A625D96EDA6A010EDA22DF50D8A4FDD050
:1007D000CF0EA625D96EDA6A010EDA22010EDF6E7F
:1007E000A65102017B19D8A435D0010E1F6E070E49
:1007F000206E200E61EC14F0010E1B6E200EEBEC4F
:1008000013F0010E1B6E200EEBEC13F0010E1B6EAD
:10081000200EEBEC13F0010E1B6E200EEBEC13F030
:10082000010E1B6E200EEBEC13F0010E1B6E200E62
:10083000EBEC13F0010E1B6E200EEBEC13F0010E2F
:100840001B6E200EEBEC13F0010E1B6E200EEBEC7A
:1008500013F0BBD0020E1F6E070E206E200E61EC4F
:1008600014F0010E1B6E200EEBEC13F0010E1B6E4C
:10087000200EEBEC13F0010E1B6E200EEBEC13F0D0
:10088000010E1B6E200EEBEC13F0010E1B6E200E02
:10089000EBEC13F0010E1B6E200EEBEC13F0010ECF
:1008A0001B6E200EEBEC13F0010E1B6E200EEBEC1A
:1008B00013F0010E1B6E200EEBEC13F086D0CF0E62
:1008C000A625D96EDA6A010EDA22000EDF6EA65175
:1008D0000E0D550EF324D96E010EF420DA6EDF50A2
:1008E0000201826F0001A6510E0D560EF324D96E3F
:1008F000010EF420DA6EDF5002017F6F0001A65175
:100900000E0D570EF324D96E010EF420DA6E01019C
:10091000DFAC02D0010E01D0000E0201806F000199
:10092000A6510E0D570EF324D96E010EF420DA6E87
:100930000101DFAA02D0010E01D0000E0201816F79
:100940000001A6510E0D570EF324D96E010EF420AE
:10095000DA6E0101DFA404D0020182513D0F826FE3
:100960000001A65102017B19D8A418D082C2E6F179
:100970007FC2E7F1000E0101E86F000EE96F80C24F
:10098000EAF181C2EBF1010EEC6F070EED6F010E83
:10099000EE6F0001A65156EC10F017D082C2E6F1BE
:1009A0007FC2E7F1000E0101E86F000EE96F80C21F
:1009B000EAF181C2EBF1020EEC6F070EED6F010E52
:1009C000EE6F0001A65156EC10F00001A62B050EAB
:1009D000A619D8A4D7D4010EA66FD4D40001F56F00
:1009E0000F0E0001F86FF551D8B411D0010EF66F5B
:1009F0009F0EF625D96EDA6A000EDA22F551DE185E
:100A0000D8B4F6C0F8F0F62B040EF665F1D70F0E49
:100A1000F819D8A4D3D128D2220EF825D96EDA6AD3
:100A2000000EDA22DFB016D09F0EF825D96EDA6AF2
:100A3000000EDA22540EF825E16EE26A010EE2227F
:100A4000DFCFE7FF220EF825D96EDA6A000EDA2230
:100A5000000EDB80BD0EF825D96EDA6A010EDA22AF
:100A600066C0DFFF130E626502D0130E626F0D0EBB
:100A7000676502D00D0E626F62C0F4F0620EF4255D
:100A8000D96EDA6A000EDA22C30EF825E16EE26A48
:100A9000010EE222DFCFE7FFF8510E0D540EF324D2
:100AA000D96E010EF420DA6E67C0DFFF010EF76F1A
:100AB0003BD0670EF725D96EDA6A000EDA22F851BC
:100AC0000E0D540EF16F010EF26FF350F127F4503A
:100AD000F223F751F125E16E000EF221E26EDE50B5
:100AE000E618D8B420D0670EF725D96EDA6A000E62
:100AF000DA22F8510E0D540EF06F010EF16FF35023
:100B0000F027F450F123F751F025E16E000EF121AA
:100B1000E26EDFCFE7FF220EF825D96EDA6A000E0B
:100B2000DA22000EDB82F72BF8510E0D540EF3245F
:100B3000D96E010EF420DA6EF751DE5CD8B0B9D769
:100B40008D0EF825D96EDA6A000EDA226CC0DFFF4E
:100B5000750EF825D96EDA6A000EDA226DC0DFFF55
:100B60003104D8A44AD0750EF825D96EDA6A000E81
:100B7000DA22DFA613D02D50D8A410D0750EF82598
:100B8000D96EDA6A000EDA22F00EDF16810EF82531
:100B9000D96EDA6A000EDA22F00EDF16750EF8252D
:100BA000D96EDA6A000EDA22DFA00DD02D50D8A45B
:100BB0000AD08484810EF825D96EDA6A000EDA2212
:100BC000060EDF1267D0750EF825D96EDA6A000EB0
:100BD000DA22DFA65FD0810EF825D96EDA6A000E20
:100BE000DA22DFA457D08494810EF825D96EDA6A10
:100BF000000EDA22000EDB844DD0750EF825D96E7A
:100C0000DA6A000EDA22DFA614D02D50D8A411D053
:100C1000750EF825D96EDA6A000EDA22F00EDF16AC
:100C2000810EF825D96EDA6A000EDA22F00EDF1690
:100C30008494750EF825D96EDA6A000EDA22DFA0E8
:100C40000ED02D50D8A40BD08484810EF825D96EF7
:100C5000DA6A000EDA22060EDF12010E1AD0750EC5
:100C6000F825D96EDA6A000EDA22DFA613D0810EDB
:100C7000F825D96EDA6A000EDA22DFA40BD084944C
:100C8000810EF825D96EDA6A000EDA22000EDB84B6
:100C9000000E2D6E220EF825D96EDA6A000EDA22C9
:100CA0007F0EDF169F0EF825D96EDA6A000EDA2263
:100CB0003B0EF825E16EE26A020EE222DFCFE7FF8B
:100CC00092D0220EF825D96EDA6A000EDA22010ED1
:100CD000DF6EE8D76451D8A402D0010E01D0000E17
:100CE000F06F6351D8A402D0010E01D0000EF015B0
:100CF000E8A079D00F0E3818D8B475D03850D8B4D1
:100D000072D038C0F8F0220EF825D96EDA6A000EDB
:100D1000DA22000EDB88080E396E930EF825D96EA4
:100D2000DA6A000EDA22000EDF6E08D0930EF82584
:100D3000D96EDA6A000EDA22B4CFDFFF930EF825FF
:100D4000D96EDA6A000EDA22DF50D8B4EFD7C90EB6
:100D5000F825D96EDA6A010EDA222F0EDF6E43D043
:100D600038C0F8F09F0EF825D96EDA6A000EDA2244
:100D7000DE506319D8A41FD0930EF825D96EDA6A15
:100D8000000EDA22DE506419D8A415D0220EF82500
:100D9000D96EDA6A000EDA22010EDF6E930EF825A4
:100DA000D96EDA6A000EDA22DF501E6EF85178EC46
:100DB00015F0000E396E000E386E15D06551BF0B60
:100DC000F06FF16BF151000AD8A40DD0F051300A48
:100DD000D8B477D7010AD8B41FD60F0AD8B47AD7B7
:100DE000010AD8B4BDD70001F85112006451D8A44B
:100DF00002D0010E01D0000EF06F6351D8A402D0D2
:100E0000010E01D0000EF015E8A0EDD70F0E381836
:100E1000D8B4E9D73850D8B4E6D738C0F8F0220EA5
:100E2000F825D96EDA6A000EDA22000EDB88080E89
:100E3000396E930EF825D96EDA6A000EDA22000EAA
:100E4000DF6E08D0930EF825D96EDA6A000EDA222A
:100E5000B4CFDFFF930EF825D96EDA6A000EDA22DE
:100E6000DF50D8A474D7EED76551BF0BF06FF16B8C
:100E7000F151000AD8A4B7D7F051300AD8B421D71D
:100E80000E0AD8B4B3D7AFD70001F26FF0D100018A
:100E9000F2510C0D000EF324D96E020EF420DA6E1E
:100EA000DF50F16FF2510E0D000EF324D96E010EDA
:100EB000F420DA6E060EDF6E990EF225D96EDA6A2C
:100EC000000EDA22DF501C6E030E1C168D0EF2256A
:100ED000D96EDA6A000EDA22DF50030B1C18D8A490
:100EE00010D1990EF225D96EDA6A000EDA22870E39
:100EF000F225E16EE26A000EE222DFCFE7FFF1AFFA
:100F000008D0870EF225D96EDA6A000EDA22000EBA
:100F1000DB8E8D0EF225D96EDA6A000EDA22DFB88A
:100F20003FD0F1BB13D0F2510E0D550EF324D96E04
:100F3000010EF420DA6EF2510E0D010EF324E16E73
:100F4000010EF420E26EDFCFE7FF0AD0F2510E0D62
:100F5000010EF324D96E010EF420DA6E000EDF6E5E
:100F6000F1B913D0F2510E0D580EF324D96E010EC3
:100F7000F420DA6EF2510E0D040EF324E16E010E30
:100F8000F420E26EDFCFE7FF35D0F2510E0D040EF4
:100F9000F324D96E010EF420DA6E000EDF6E2AD033
:100FA000F2510E0D550EF324D96E010EF420DA6EB7
:100FB000F2510E0D010EF324E16E010EF420E26EEB
:100FC000DFCFE7FF990EF225D96EDA6A000EDA223A
:100FD000870EF225E16EE26A000EE222DFCFE7FF24
:100FE000F1AFD3D7870EF225D96EDA6A000EDA2276
:100FF000000EDB8E8D0EF225D96EDA6A000EDA2233
:10100000DFAA16D0990EF225D96EDA6A000EDA221E
:10101000870EF225E16EE26A000EE222DFCFE7FFE3
:10102000870EF225D96EDA6A000EDA22000EDB8E08
:101030008D0EF225D96EDA6A000EDA22DFAC16D0F8
:10104000990EF225D96EDA6A000EDA22870EF225A1
:10105000E16EE26A000EE222DFCFE7FF870EF225A3
:10106000D96EDA6A000EDA22000EDB8EF2510E0D16
:10107000030EF324D96E010EF420DA6E0101DFAC09
:1010800014D0220E0001F225D96EDA6A000EDA229F
:10109000000EDB8CF2510E0D010EF324D96E010E01
:1010A000F420DA6E000EDB8C09D0220E0001F2254E
:1010B000D96EDA6A000EDA22BF0EDF16F2510E0D7B
:1010C000560EF324D96E010EF420DA6EF2510E0D95
:1010D000020EF324E16E010EF420E26EDFCFE7FF93
:1010E000F2510E0D570EF324D96E010EF420DA6E74
:1010F000F2510E0D030EF324E16E010EF420E26EA8
:101100004FD0F2510E0D550EF324D96E010EF4207E
:10111000DA6EF2510E0D010EF324E16E010EF42091
:10112000E26EDFCFE7FFF2510E0D560EF324D96EBB
:10113000010EF420DA6EF2510E0D020EF324E16E70
:10114000010EF420E26EDFCFE7FFF2510E0D030E29
:10115000F324D96E010EF420DA6EF2510E0D570E03
:10116000F324E16E010EF420E26EE750040BDF6E13
:10117000F2510E0D040EF324D96E010EF420DA6E36
:10118000000EDF6E990EF225D96EDA6A000EDA22B1
:10119000000EDB82870EF225E16EE26A000EE2228B
:1011A000DFCFE7FF3104D8A417D0F1B70BD0000E82
:1011B0002D6E810EF225D96EDA6A000EDA22FD0E4E
:1011C000DF160AD0010E2D6E810EF225D96EDA6A75
:1011D000000EDA22000EDB82870EF225D96EDA6A63
:1011E000000EDA22F2510E0D050EF324E16E010E0F
:1011F000F420E26EDFCFE7FF810EF225D96EDA6AC6
:10120000000EDA22F2510E0D060EF324E16E010EED
:10121000F420E26EDFCFE7FF1200010E0001F06F55
:10122000F2510E0D540E1C6E010E1D6EF3501C2655
:10123000F4501D22F0511C24D96E000E1D20DA6ED0
:10124000F2510E0D000E1E6E010E1F6EF3501E2683
:10125000F4501F22F0511E24E16E000E1F20E26E9A
:10126000DFCFE7FFF02B060EF065DAD712001B5038
:10127000230AD8B40CD60B0AD8B412004B0AD8A44F
:101280001200CBD7086EEDD108500C0D000EF324E0
:10129000D96E020EF420DA6EDF50076E08500E0D84
:1012A000000EF324D96E010EF420DA6E060EDF6E06
:1012B000990E0824D96EDA6A000EDA22DF50026E27
:1012C000030E02168D0E0824D96EDA6A000EDA2299
:1012D000DF50030B0218D8A40FD1990E0824D96E41
:1012E000DA6A000EDA22870E0824E16EE26A000E46
:1012F000E222DFCFE7FF07AE08D0870E0824D96EC1
:10130000DA6A000EDA22000EDB8E8D0E0824D96E0A
:10131000DA6A000EDA220001DFB83FD007BA13D034
:1013200008500E0D550EF324D96E010EF420DA6E1E
:1013300008500E0D010EF324E16E010EF420E26E52
:10134000DFCFE7FF0AD008500E0D010EF324D96E4F
:10135000010EF420DA6E000EDF6E07B813D00850CD
:101360000E0D580EF324D96E010EF420DA6E0850DB
:101370000E0D040EF324E16E010EF420E26EDFCFB9
:10138000E7FF35D008500E0D040EF324D96E010E80
:10139000F420DA6E000EDF6E2AD008500E0D550EC6
:1013A000F324D96E010EF420DA6E08500E0D010EF2
:1013B000F324E16E010EF420E26EDFCFE7FF990E19
:1013C0000824D96EDA6A000EDA22870E0824E16E4C
:1013D000E26A000EE222DFCFE7FF07AED3D7870E27
:1013E0000824D96EDA6A000EDA22000EDB8E8D0E2A
:1013F0000824D96EDA6A000EDA22DFAA16D0990E16
:101400000824D96EDA6A000EDA22870E0824E16E0B
:10141000E26A000EE222DFCFE7FF870E0824D96ED2
:10142000DA6A000EDA22000EDB8E8D0E0824D96EE9
:10143000DA6A000EDA22DFAC16D0990E0824D96ED3
:10144000DA6A000EDA22870E0824E16EE26A000EE4
:10145000E222DFCFE7FF870E0824D96EDA6A000E9A
:10146000DA22000EDB8E08500E0D030EF324D96E27
:10147000010EF420DA6E0101DFAC13D0220E082435
:10148000D96EDA6A000EDA22000EDB8C08500E0DDF
:10149000010EF324D96E010EF420DA6E000EDB8CFF
:1014A00008D0220E0824D96EDA6A000EDA22BF0EA6
:1014B000DF1608500E0D560EF324D96E010EF420DF
:1014C000DA6E08500E0D020EF324E16E010EF420C8
:1014D000E26EDFCFE7FF08500E0D570EF324D96EF2
:1014E000010EF420DA6E08500E0D030EF324E16EA7
:1014F000010EF420E26E4FD008500E0D550EF3246D
:10150000D96E010EF420DA6E08500E0D010EF32490
:10151000E16E010EF420E26EDFCFE7FF08500E0D02
:10152000560EF324D96E010EF420DA6E08500E0D1B
:10153000020EF324E16E010EF420E26EDFCFE7FF2E
:1015400008500E0D030EF324D96E010EF420DA6E4E
:1015500008500E0D570EF324E16E010EF420E26EDA
:10156000E750040BDF6E08500E0D040EF324D96E05
:10157000010EF420DA6E000EDF6E990E0824D96E8B
:10158000DA6A000EDA22000EDB82870E0824E16E92
:10159000E26A000EE222DFCFE7FF3104D8A417D0C1
:1015A00007B60BD0000E2D6E810E0824D96EDA6AB4
:1015B000000EDA22FD0EDF160AD0010E2D6E810E0E
:1015C0000824D96EDA6A000EDA22000EDB82870E5A
:1015D0000824D96EDA6A000EDA2208500E0D050EC4
:1015E000F324E16E010EF420E26EDFCFE7FF810EFF
:1015F0000824D96EDA6A000EDA2208500E0D060EA3
:10160000F324E16E010EF420E26EDFCFE7FF12005B
:10161000010E066E08500E0D540E026E010E036E82
:10162000F3500226F450032206500224D96E000E15
:101630000320DA6E08500E0D000E046E010E056ECA
:10164000F3500426F450052206500424E16E000EE7
:101650000520E26EDFCFE7FF062A060E0664DAD722
:1016600012000150230AD8B40FD60B0AD8B41200C6
:101670004B0AD8A41200CCD70E01C89194A442D032
:1016800091CF14F03650D8A424D0D8901430146ED2
:1016900014500001A019D8A402D0010E13D0145088
:1016A000A119D8A402D0020E0DD01450A219D8A4AA
:1016B00002D0030E07D01450A319D8A402D0040EF0
:1016C00001D0000E356E010E336E34508109346E38
:1016D000349894AA02D096BC5AD035500C0D3C0ECA
:1016E000126E020E136EF3501226F450132236506F
:1016F0001224D96E000E1320DA6EDF50916E362A56
:10170000348C45D094BA25D091CF14F0D8901430B1
:10171000146E000E366E14500001A019D8A402D029
:10172000010E13D01450A119D8A402D0020E0DD06E
:101730001450A219D8A402D0030E07D01450A31934
:10174000D8A402D0040E01D0000E356E010E326E08
:101750001ED094B81CD091CF14F035500C0D000E53
:10176000126E020E136EF3501226F45013223650EE
:101770001224D96E000E1320DA6E14C0DFFF362A51
:1017800036C0C4F0010E316E990E0001C36F95880A
:10179000978C000E0001C26F94A81200979C000E57
:1017A000366E010EC26F3304D8A424D03F0E341617
:1017B000348A000E336E220E3524D96EDA6A000E9A
:1017C000DA22DFA208D0220E3524D96EDA6A000EA2
:1017D000DA22000EDB8ED50E3524D96EDA6A010EC0
:1017E000DA22DB0E3524E16EE26A010EE222DFCF5F
:1017F000E7FF12003204D8A41200349A3488000E95
:10180000326EDB0E3524D96EDA6A010EDA22990EB9
:101810003524E16EE26A000EE222DFCFE7FF3950A5
:10182000D8B426D039A616D0930E3824D96EDA6AE9
:10183000000EDA22DF500C6E2F0E0D6E000E0E6EB3
:101840009F0E3824D96EDA6A000EDA22DF504EEC91
:101850000DF00BD039A409D0000E0C6E2E0E0D6EBB
:10186000000E0E6E000E4EEC0DF0000E396E1200E2
:101870003550D8A414D0040E376403D0010E376E4F
:1018800001D0372A930E3724D96EDA6A000EDA2295
:10189000DF50D8B412003750D1EC0FF01200220EF6
:1018A0003524D96EDA6A000EDA22DF50820B820A02
:1018B000D8A415D0220E3524D96EDA6A000EDA22A9
:1018C0007D0EDF16930E3524D96EDA6A000EDA2209
:1018D000DF50D8B412003550D1EC0FF01200040ED6
:1018E000376403D0010E376E01D0372A930E3724A8
:1018F000D96EDA6A000EDA22DF50D8B412003750FF
:10190000D1EC0FF012000001F96FF5C01BF00001DF
:10191000F95138EC15F00001FA6FF69DB4D0F9C01A
:10192000E2F0F5C0E3F0210EE46F2D04D8B4E48DAD
:10193000F7C0E5F0000EE66F050E2C6E0F0EFA19DB
:10194000D8B446D0230E1B6EFA5144EC07F0060EB5
:101950000001E66FFA510E0D010EF324D96E010E4F
:10196000F420DA6EDF50E76FFA510E0D020EF32409
:10197000D96E010EF420DA6EDF50E86FFA510E0DC9
:10198000030EF324D96E010EF420DA6EDF50E96FF6
:10199000FA510E0D040EF324D96E010EF420DA6E06
:1019A000DF50EA6FFA510E0D050EF324D96E010EC9
:1019B000F420DA6EDF50EB6FFA510E0D060EF324B1
:1019C000D96E010EF420DA6EDF50EC6F0B0E2C6E28
:1019D000E20EF06F000EF16F2CC0F2F0000ED0ECB2
:1019E00012F00001F86F7B0EFA25D96EDA6A000E4C
:1019F000DA22DF2AF8C01BF0CD511FEC16F01200DE
:101A0000F9C0E2F0F5C0E3F02F0EE46F000EE56FD1
:101A1000040E2C6EE20EF06F000EF16F2CC0F2F08F
:101A2000000ED0EC12F00001F86F3988F8C01BF0FE
:101A3000CD511FEC16F01200F9C0E2F0F5C0E3F052
:101A40002E0EE46F000EE56F000EE66F050E2C6E95
:101A5000080E396EE2C0B2F0E3C0B1F0E4C0B0F0FD
:101A6000E5C0AFF0E20EF06F000EF16F2CC0F2F0A7
:101A7000000ED0EC12F00001F86FF8C01BF0CD5151
:101A80001FEC16F01200F651210AD8B448D70F0AFD
:101A9000D8B4D2D7010AD8A41200B2D7106E0CC0A5
:101AA00001F0105058EC15F0116E0D9CB7D010C01D
:101AB000E2F00CC0E3F0210E0001E46F2D04D8B475
:101AC000E48D0EC0E5F0000EE66F050E2C6E0F0ED5
:101AD0001118D8B446D0230E016E115042EC09F013
:101AE000060E0001E66F11500E0D010EF324D96EA3
:101AF000010EF420DA6EDF50E76F11500E0D020E6A
:101B0000F324D96E010EF420DA6EDF50E86F115025
:101B10000E0D030EF324D96E010EF420DA6EDF50A1
:101B2000E96F11500E0D040EF324D96E010EF4204E
:101B3000DA6EDF50EA6F11500E0D050EF324D96EE8
:101B4000010EF420DA6EDF50EB6F11500E0D060E11
:101B5000F324D96E010EF420DA6EDF50EC6F0B0E19
:101B60002C6EE20E066E000E076E2CC008F0000E02
:101B700005EC13F00F6E7B0E1124D96EDA6A000E9D
:101B8000DA22DF2A0FC001F00001CD5130EC16F04F
:101B9000120010C0E2F00CC0E3F02F0E0001E46F61
:101BA000000EE56F040E2C6EE20E066E000E076E40
:101BB0002CC008F0000E05EC13F00F6E39880FC032
:101BC00001F00001CD5130EC16F0120010C0E2F02F
:101BD0000CC0E3F02E0E0001E46F000EE56F000E66
:101BE000E66F050E2C6E080E396EE2C0B2F0E3C04F
:101BF000B1F0E4C0B0F0E5C0AFF0E20E066E000E4A
:101C0000076E2CC008F0000E05EC13F00F6E0FC02D
:101C100001F00001CD5130EC16F012000D50210AF8
:101C2000D8B445D70F0AD8B4D1D7010AD8A4120026
:101C3000B0D71E6E98D01E500E0D550EF324D96EDF
:101C4000010EF420DA6EDF500101A86F1E500E0D58
:101C5000560EF324D96E010EF420DA6EDF50FC0B21
:101C6000A96F1E500C0D3D0EF324D96E020EF42008
:101C7000DA6EDF501C6EFC0E1C161E500E0D560E3A
:101C8000F324D96E010EF420DA6EDF50FC0B1C1821
:101C9000D8A4A9831E500E0D570EF324D96E010E41
:101CA000F420DA6EDF50AA6F1E500C0D3E0EF324A6
:101CB000D96E020EF420DA6E1E500E0D570EF3246C
:101CC000E16E010EF420E26EDE50E618D8B40AD0C0
:101CD0001E500E0D570EF324D96E010EF420DA6E4D
:101CE000DFAEA9811E500E0D580EF324D96E010EE1
:101CF000F420DA6EDF50AB6F1E500C0D3C0EF32457
:101D0000D96E020EF420DA6EA8C1DFFF1E500C0D52
:101D10003D0EF324D96E020EF420DA6EA9C1DFFF66
:101D20001E500C0D3E0EF324D96E020EF420DA6E16
:101D3000AAC1DFFF1E500C0D3F0EF324D96E020E18
:101D4000F420DA6EABC1DFFF8D0E1E24D96EDA6A85
:101D5000000EDA22D50E1E24E16EE26A010EE222A6
:101D6000DFCFE7FF12001B50220AD8B464D7010A64
:101D70001200010E1B6E020EC1EC13F02A0E216E32
:101D80008E0EE82EFED7212EFCD7010E1B6E480EBC
:101D9000EBEC13F0010E1B6E520EEBEC13F0010E88
:101DA0001B6E580EEBEC13F0010E1B6E2D0EEBECC0
:101DB00013F0010E1B6E490EEBEC13F0010E1B6EBF
:101DC0006E0EEBEC13F0010E1B6E740EEBEC13F0C9
:101DD000010E1B6E650EEBEC13F0010E1B6E720E06
:101DE000EBEC13F0010E1B6E660EEBEC13F0010E24
:101DF0001B6E610EEBEC13F0010E1B6E630EEBEC31
:101E000013F0010E1B6E650EEBEC13F0010E1B6E52
:101E1000200EEBEC13F0020E1F6E010E206E200E52
:101E200061EC14F0010E1B6E560EEBEC13F0010E7C
:101E30001B6E650EEBEC13F0010E1B6E720EEBECDD
:101E400013F0010E1B6E730EEBEC13F0010E1B6E04
:101E5000690EEBEC13F0010E1B6E6F0EEBEC13F042
:101E6000010E1B6E6E0EEBEC13F0010E1B6E200EBE
:101E7000EBEC13F0010E1B6E310EEBEC13F0010EC8
:101E80001B6E2E0EEBEC13F0010E1B6E310EEBEC05
:101E900013F012000001F66F9F0E0001F625D96EB7
:101EA000DA6A000EDA22DF50E26F930EF625D96E61
:101EB000DA6A000EDA22DF50E36F210EE46F2D04A0
:101EC000D8B4E48DC30EF625D96EDA6A010EDA2293
:101ED000DF50E56F230E1B6EF65144EC07F0060E43
:101EE0000001E66FF6510E0D010EF324D96E010EBE
:101EF000F420DA6EDF50E76FF6510E0D020EF32478
:101F0000D96E010EF420DA6EDF50E86FF6510E0D37
:101F1000030EF324D96E010EF420DA6EDF50E96F60
:101F2000F6510E0D040EF324D96E010EF420DA6E74
:101F3000DF50EA6FF6510E0D050EF324D96E010E37
:101F4000F420DA6EDF50EB6FF6510E0D060EF3241F
:101F5000D96E010EF420DA6EDF50EC6F0B0E2C6E92
:101F6000E20EF06F000EF16F2CC0F2F0000ED0EC1C
:101F700012F00001F56F7B0EF625D96EDA6A000EBD
:101F8000DA22DF2AF5C01BF0CD511FEC16F0870EC8
:101F90000001F625D96EDA6A000EDA22000EDF6E35
:101FA00012000D6E9F0E0D24D96EDA6A000EDA2231
:101FB000DF500001E26F930E0D24D96EDA6A000E35
:101FC000DA22DF50E36F210EE46F2D04D8B4E48DE4
:101FD000C30E0D24D96EDA6A010EDA22DF50E56FE6
:101FE000230E016E0D5042EC09F0060E0001E66F63
:101FF0000D500E0D010EF324D96E010EF420DA6E91
:10200000DF50E76F0D500E0D020EF324D96E010E56
:10201000F420DA6EDF50E86F0D500E0D030EF3243E
:10202000D96E010EF420DA6EDF50E96F0D500E0DFF
:10203000040EF324D96E010EF420DA6EDF50EA6F3D
:102040000D500E0D050EF324D96E010EF420DA6E3C
:10205000DF50EB6F0D500E0D060EF324D96E010EFE
:10206000F420DA6EDF50EC6F0B0E2C6EE20E066E73
:10207000000E076E2CC008F0000E05EC13F00C6E7D
:102080007B0E0D24D96EDA6A000EDA22DF2A0CC02C
:1020900001F00001CD5130EC16F0870E0D24D96E01
:1020A000DA6A000EDA22000EDF6E12000001FA6F0B
:1020B000ECC120F0EDC121F0070EACEC14F00001F2
:1020C000FA51020FA0EC16F0010E1B6E3A0EEBEC6B
:1020D00013F0010E1B6E4C0EEBEC13F00101E651F8
:1020E0001AEC11F0300E4318D8B406D0010E1B6E56
:1020F0004350EBEC13F005D0010E1B6E200EEBEC01
:1021000013F0010E1B6E4250EBEC13F00101E7A53A
:1021100006D0010E1B6E520EEBEC13F005D0010E33
:102120001B6E560EEBEC13F00101E739E8461F0B6E
:102130001AEC11F0300E4318D8B406D0010E1B6E05
:102140004350EBEC13F005D0010E1B6E200EEBECB0
:1021500013F0010E1B6E4250EBEC13F00101EB513A
:10216000D8B408D0ECC11FF0100E206E210E61EC27
:1021700014F01200ECC11FF0100E206E200E61EC66
:1021800014F01200090E206E1E0E1F6EE40EE82ED3
:10219000FED71F2EFCD7202EFAD700D0000E1B6EC4
:1021A000380EC1EC13F0B60E00D000D0E82EFCD7EC
:1021B00000D000D000D0000E1B6E380EC1EC13F022
:1021C000B60E00D000D0E82EFCD700D000D000D052
:1021D000010E1B6E0C0EC1EC13F0B60E00D000D039
:1021E000E82EFCD700D000D000D0010E1B6E010EEF
:1021F000C1EC13F02A0E1F6E8E0EE82EFED71F2E96
:10220000FCD7010E1B6E060EC1EC13F02A0E1F6EDA
:102210008E0EE82EFED71F2EFCD7010E1B6E020E6F
:10222000C1EC13F02A0E1F6E8E0EE82EFED71F2E65
:10223000FCD71200216E21C01BF01C6A000E1E6E1E
:10224000640E1D6E60EC12F01B50436E43C01BF019
:102250001C6A000E1E6E0A0E1D6E60EC12F01B5002
:10226000426E4250435C0001F06FF16BD8A0F10761
:10227000000EF36F0A0EF26F6CEC11F00001F051DA
:10228000436E43C01BF01C6AFF0E1E6EF60E1D6EE1
:102290000CEC16F021500001F86FF96B1B50F82779
:1022A0001C50F9234250F85DF06FF951D8A0F905A0
:1022B000F16F000EF36F640EF26F6CEC11F0000121
:1022C000F051446E4450300F446E4350300F436E13
:1022D0004250300F426E1200000E0001F56FF3AF56
:1022E00006D0F26DF31FD8B0F32B010EF56FF1AFEE
:1022F00006D0F06DF11FD8B0F12B010EF51B000ECA
:10230000F76F000EF66FF251F311D8B41CD0010E26
:10231000F46F04D0D890F237F337F42BF3AFFAD739
:10232000D890F637F737F251F05DF351F159D8A054
:1023300005D0F251F05FF351F15BF681D890F333A1
:10234000F233F42FEDD7F551D8B404D0F66DF71F62
:10235000D8B0F72BF6C0F0F0F7C0F1F01200000E85
:102360001F6E220E1F24D96EDA6A000EDA22000ECA
:10237000DF6E9F0E1F24D96EDA6A000EDA221F501C
:10238000480FDF6E1F50580F94EC16F05A0AD8A46D
:102390000BD0930E1F24D96EDA6A000EDA221F507A
:1023A000480F94EC16F007D0930E1F24D96EDA6A0A
:1023B000000EDA22000EDF6E1F2A040E1F64D1D732
:1023C000010E94EC16F00B0AD8B412000B0E1B6E23
:1023D000010E95EC15F01200980EF66E2D0EF76EAC
:1023E000000EF86E0900F5CFFDF00900F5CFFEF004
:1023F000860EF66E2D0EF76E000EF86E00EE40F0B3
:1024000010EE05F00900F5CFEEFFE550E150FAE1DE
:1024100002EE00F0780EEE6AE806FDE101EE00F053
:10242000E60EEE6AE806FDE100EE60F0900EEE6A60
:10243000E806FDE100EE22F01E0EEE6AE806FDE180
:1024400045904592000EF86E00013BEF00F00F0E34
:10245000216E29D06351EEEC04F0216E0F0E21188D
:10246000D8B429D07B0E2124D96EDA6A000EDA2284
:10247000DF50D8B407D07B0E2124D96EDA6A000E63
:10248000DA22DF067B0E2124D96EDA6A000EDA2208
:10249000DF50D8B410D07B0E2124D96EDA6A000E3A
:1024A000DA22DF0608D000016151400AD8B403D017
:1024B000C10AD8B4CFD7000E0001CB6F2150120053
:1024C000000E206E1CAE06D01B6C1C1ED8B01C2A41
:1024D000010E206E1EAE04D01D6C1E1ED8B01E2A2A
:1024E0001D501E10D8B418D0010E1F6E04D0D89005
:1024F0001D361E361F2A1EAEFAD71D501B5C1E50FD
:102500001C58D8A004D01D501B5E1E501C5AD890D9
:102510001E321D321F2EF1D72050D8B404D01B6CB0
:102520001C1ED8B01C2A1BC01BF01CC01CF01200C3
:10253000000EB46E010E0001CC6F9CA202D09C98DC
:102540009C888282600E3D24D96EDA6A000EDA22FF
:1025500098CFDFFF3D2A140E3D6402D0000E3D6E81
:10256000030E3D18D8B462C03FF03D50016E026AC0
:102570003F50036E046A040E0326000E042201502D
:1025800003180BE102500418D8A407D0010ECB6F3A
:10259000000ECC6F3DC0C8F01200000ECB6F1200D1
:1025A0000001F36F020E0001CD6FF3C0CEF0F2C058
:1025B000CFF0000EF46F0FD0F451F025D96E000E5D
:1025C000F121DA6ED00EF425E16EE26A000EE2220D
:1025D000DFCFE7FFF42BF251F45DD8A0EDD7CD0E9D
:1025E0001B6E000E1C6EF451020F1D6EE2EC15F016
:1025F000206ED00E0001F425D96EDA6A000EDA22C0
:1026000020C0DFFFF451030F12000A6E020E00011A
:10261000CD6F0AC0CEF008C0CFF0000E0B6E0FD009
:102620000B500624D96E000E0720DA6ED00E0B2454
:10263000E16EE26A000EE222DFCFE7FF0B2A0850CC
:102640000B5CD8A0EDD7CD0E016E000E026E0B50C4
:10265000020F036EF7EC15F0096ED00E0B24D96E45
:10266000DA6A000EDA2209C0DFFF0B50030F1200F6
:10267000000E826E000E836E000E846EFC0E876E5E
:10268000000E886E1A0E896EE00E0F011C6F146921
:10269000FC0E0C6F000E286F000E136F010E0B6FF7
:1026A000000E1B6F000E0A6F000E126F000E1A6FE5
:1026B000096911691969090E0E01F26F110EB06FE7
:1026C000140EB36F0D0EF56F0E0EF66F130EB26F84
:1026D00012000001FA6F0001FA511AEC11F0300EED
:1026E0004418D8A406D0010E1B6E200EEBEC13F09C
:1026F00005D0010E1B6E4450EBEC13F0300E441865
:10270000D8A40AD0300E4318D8A406D0010E1B6EF0
:10271000200EEBEC13F005D0010E1B6E4350EBECDA
:1027200013F0010E1B6E4250EBEC13F012000E0181
:10273000C09B300E1B6E250E1C6EBEEC16F00E01FB
:10274000C099640E1B6E2B0E1C6EB9EC16F0080EB1
:102750009E6E900E9C6E240E9D6E8A0E9A6E000EDA
:102760009B6E000E3E6E000E0001C76F000E3C6EA9
:10277000000E3D6E000E3B6E000E3A6E0E01C08BD9
:1027800012001C6E1B04D8A41DD0B60E00D000D0C1
:10279000E82EFCD700D000D000D0849C8868000EC2
:1027A0001E6E849A848C848E8DCF1DF0849E1DBEF7
:1027B00002D01D0E1E6E1E2A1D0E1E64F2D7849CB2
:1027C000000E886E000E886E849C849A1CC083FF65
:1027D000848E849E12001C6E1B04D8A41DD0B60EDD
:1027E00000D000D0E82EFCD700D000D000D0849CD0
:1027F0008868000E1E6E849A848C848E8DCF1DF0A6
:10280000849E1DBE02D01D0E1E6E1E2A1D0E1E644D
:10281000F2D7849C000E886E849C848A1CC083FF3F
:10282000848E849E12000F0E0001F06F000EF16F77
:10283000F1512608D96E000ED8A0E82A0008DA6EF9
:10284000DF50D8A411D0000E1E6EF151040878ECB0
:1028500015F0000E1E6E0001F151140878EC15F011
:102860000001F1510408F06FF12B030EF165E0D780
:10287000F05112000101E66F0001FB05D8B404D04D
:10288000020EFB19D8A41200FB07FC51D8B41200A9
:10289000110EFC611200FC07FB51400DF350800F3C
:1028A0000101E76FE7510001FC250101E76F010E0F
:1028B0001B6EE751C1EC13F00101E65169EC13F016
:1028C00012000001F06F1F04D8B404D0020E1F18CC
:1028D000D8A412001F062050D8B41200110E206098
:1028E000120020061F50400DF350800F0001F16FC1
:1028F000F1512024F16F010E1B6EF151C1EC13F068
:10290000010E1B6E0001F051EBEC13F01200000EF3
:102910001B6E000E306E010E1C6E220E1C24D96E32
:10292000DA6A000EDA22DF50D8B408D0302A1B5001
:10293000D8A404D01CC02FF0010E1B6E1C2A040E5C
:102940001C64EBD7020E306402D0010E01D0000EE1
:102950000001BB6F2F5012000001F06F2004D8B4AB
:1029600004D0020E2018D8A4120020062150D8B49A
:102970001200110E2160120021062050400DF3506C
:10298000800F0001F16FF1512124F16F010E1B6ED8
:10299000F151C1EC13F00001F051A0EC16F012005F
:1029A0000F0E1B6E000E1C6E1C502608D96E000EFA
:1029B000D8A0E82A0008DA6EDF50D8A40ED01C5048
:1029C0009708D96E000ED8A0E82A0008DA6EDF500A
:1029D000D8A403D01C5004081B6E1C2A030E1C64D0
:1029E000E3D71B5012000E01C9A312002B28D8A454
:1029F00003D0000E2B6E01D02B2A0001AB51D8A4BE
:102A0000AB07AA51D8A4AA07A951D8A4A907A851CD
:102A1000D8A4A807C351D8A4C3072A50D8A42A060B
:102A2000A751D8A4A7070E01C99312002EC021F008
:102A30003450D8B408D02E50D8A402D0010E01D002
:102A4000000E2E6E02D0000E216E2150D8B408D098
:102A5000020E1F6E020E206E2A0E61EC14F01200A0
:102A6000020E1F6E020E206E200E61EC14F012009A
:102A70001D6E0F0E1E6E010E1F6E9F0E1F24D96E4F
:102A8000DA6A000EDA221D50DE18D8A40BD0930E9D
:102A90001F24D96EDA6A000EDA221B50DE18D8B471
:102AA0001FC01EF01F2A040E1F64E7D71E5012001D
:102AB000036E0F0E046E010E056E9F0E0524D96E77
:102AC000DA6A000EDA220350DE18D8A40BD0930E77
:102AD0000524D96EDA6A000EDA220150DE18D8B465
:102AE00005C004F0052A040E0564E7D7045012005F
:102AF0001F6E1F50480F206E2050100F94EC16F0E0
:102B00005A0AD8B406D05A0E1B6E2050100F95ECFE
:102B100015F0205094EC16F01E18D8B412001EC008
:102B20001BF0205095EC15F012001C6E000EF2BE4A
:102B3000010E1D6E1CC079FF000E7A6E310E7B6E89
:102B40001BC07CFF7F8EF29E550E816EAA0E816E99
:102B5000808880B8FED71DB002D0F29E01D0F28EE0
:102B60007F9E12003C50D8B40FD0CD0E3E24D96EBB
:102B7000DA6A000EDA22DF50996E3E2A140E3E64A5
:102B80000AD0150E3E6E07D00E01C099000E00014E
:102B9000CA6F000E3D6E3C061200010EB86E000EAC
:102BA000B76E000EB96EB568000EB46E0E01C9970F
:102BB000C187000E1B6E000E1C6EB4EC16F0D00E1A
:102BC000B66E1200000E1E6E000E1F6E0AD01F5051
:102BD0001B24D96E000E1C20DA6EDF501E181E6EEC
:102BE0001F2A1F501D5CD8B0F2D71E501200000ED5
:102BF000046E000E056E0AD005500124D96E000E39
:102C00000220DA6EDF500418046E052A0550035CBA
:102C1000D8B0F2D7045012001B501D02F3CF1FF0A2
:102C2000F4CF20F01B501E02F35020261C501D0232
:102C3000F35020261FC01BF020C01CF012001C6E99
:102C4000010E0001CA6F1BC0C9F01BC03CF00E0191
:102C5000C0B904D01CC099FF010E3E6EC08912009D
:102C6000026E010E0001CA6F01C0C9F001C03CF044
:102C70000E01C0B904D002C099FF010E3E6EC0899A
:102C80001200000E946E260E956E010E966E400E8A
:102C9000976EF00E936E900E926E0E01C891C081E9
:102CA0001200CAEC16F06EEC16F038EC13F088EC5B
:102CB00016F0CDEC15F060EC16F097EC13F0120066
:102CC000050EBE6E000EBD6E000EBF6EBB68000E20
:102CD000BA6E0E01C993A00EBC6E1200000E0E015A
:102CE000DC6F000EDD6F000EDE6F000EDF6F000E7A
:102CF000E06F000EE16F1200D0EC14F0216E0F0EA9
:102D00002118D8A403D013EC14F0216E2150120026
:102D1000600E0E01D36F000ED56F000ED76F080E38
:102D2000D96F000ED86F12001B6E1BC079FF000E0A
:102D30007A6E310E7B6E808000F000F07C501200C5
:102D40001F6E010E1B6E1F50300FEBEC13F01200C4
:102D5000010E1B6E010EC1EC13F012000E01C9979B
:102D6000000E3D6E829212001BC0F1F11CC0F2F108
:102D700012001BC0F5F11CC0F6F112001BC0F3F1EC
:102D80001CC0F4F112002020202020FFB68E12007B
:102D9000BC8E1200F29A12000F0EFFFFFFFFFFFF22
:102DA000FFFFFFFFFFFFFFFFFFFFFFFFFFFFFFFF33
:102DB000FFFFFFFFFFFFFFFFFFFFFFFFFFFFFFFF23
:102DC000FFFFFFFFFFFFFFFFFFFFFFFFFFFFFFFF13
:102DD000FFFFFFFFFFFFFFFFFFFFFFFFFFFFFFFF03
:020000040030CA
:0C0000008CFFFFFF9FFFFFFFFFFFFFFFD3
:020000040020DA
:10000000FFFFFFFFFFFFFFFFFFFFFFFFFFFFFFFF00
:10001000FFFFFFFFFFFFFFFFFFFFFFFFFFFFFFFFF0
:10002000FFFFFFFFFFFFFFFFFFFFFFFFFFFFFFFFE0
:10003000FFFFFFFFFFFFFFFFFFFFFFFFFFFFFFFFD0
:10004000FFFFFFFFFFFFFFFFFFFFFFFFFFFFFFFFC0
:10005000FFFFFFFFFFFFFFFFFFFFFFFFFFFFFFFFB0
:10006000FFFFFFFFFFFFFFFFFFFFFFFFFFFFFFFFA0
:10007000FFFFFFFFFFFFFFFFFFFFFFFFFFFFFFFF90
:10008000FFFFFFFFFFFFFFFFFFFFFFFFFFFFFFFF80
:10009000FFFFFFFFFFFFFFFFFFFFFFFFFFFFFFFF70
:1000A000FFFFFFFFFFFFFFFFFFFFFFFFFFFFFFFF60
:1000B000FFFFFFFFFFFFFFFFFFFFFFFFFFFFFFFF50
:1000C000FFFFFFFFFFFFFFFFFFFFFFFFFFFFFFFF40
:1000D000FFFFFFFFFFFFFFFFFFFFFFFFFFFFFFFF30
:1000E000FFFFFFFFFFFFFFFFFFFFFFFFFFFFFFFF20
:1000F000FFFFFFFFFFFFFFFFFFFFFFFFFFFFFFFF10
:020000040031C9
:10000000FF0BFFFFFFFFFFFFFFFFFFFFFFFFFFFFF4
:10001000FFFFFFFFFFFFFFFFFFFFFFFFFFFFFFFFF0
:10002000FFFFFFFFFFFFFFFFFFFFFFFFFFFFFFFFE0
:10003000FFFFFFFFFFFFFFFFFFFFFFFFFFFFFFFFD0
:10004000FFFFFFFFFFFFFFFFFF00000807FFFFFFAD
:10005000FFFFFFFFFFFFFFFFFF00005A5AFFFFFFF8
:10006000FFFFFFFFFFFFFFFFFF5A5AFFFFFFFFFFEA
:10007000FFFFFFFFFFFFFFFFFFFFFFFFFFFFFFFF90
:10008000FFFFFFFFFFFFFFFFFFFFFFFFFFFFFFFF80
:10009000FFFFFFFFFFFFFFFFFFFFFFFFFFFFFFFF70
:1000A000FFFFFFFFFFFFFFFFFFFFFFFFFFFFFFFF60
:1000B000FFFFFFFFFFFFFFFFFFFFFFFFFFFFFFFF50
:1000C000FFFFFFFFFFFFFFFFFFFFFFFFFFFFFFFF40
:1000D000FFFFFFFFFFFFFFFFFFFFFFFFFFFFFFFF30
:1000E000FFFFFFFFFFFFFFFFFFFFFFFFFFFFFFFF20
:1000F000FFFFFFFFFFFFFFFFFFFFFFFFFFFFFFFF10
:00000001FF
